:100000000C9464000C9481000C9481000C94810089
:100010000C9481000C9481000C9481000C9481005C
:100020000C9481000C9481000C94FC030C948100CE
:100030000C9481000C9481000C9481000C9481003C
:100040000C9481000C9481000C9481000C9481002C
:100050000C9481000C9481000C945B01510A802A5D
:100060000000000A00FF000059551801111E111B65
:10007000500B411B411F1101511F511B000000007B
:1000800000000000000000000000510F91394114F1
:100090009131411E410E411D500F802010154886A0
:1000A0004014780570855115510E5195518E21904F
:1000B00081205015484450C528C028200950000010
:1000C000000000000000000011241FBECFEFD4E0AC
:1000D000DEBFCDBF11E0A0E0B1E0E4EFF0E102C08F
:1000E00005900D92A235B107D9F711E0A2E5B1E074
:1000F00001C01D92A33AB107E1F70E94DA030C9404
:1001000078080C940000DF92EF92FF920F931F93F8
:10011000D82E80937C0041E0841751F480917C00BC
:10012000806C80937C002B99FECF2B9BFECF0AC066
:1001300080917C00806480937C0080917C008F772C
:1001400080937C0083E880937A0080917A008064B9
:1001500080937A0080917A0084FFFCCF2091870100
:100160003091880160E0EE24FF2487011AC080915D
:100170007A00806480937A0080917A0084FFFCCFBB
:100180009091780080917900F82FE0E0AF01490F5D
:10019000511DCA01A0E0B0E0E80EF91E0A1F1B1FA6
:1001A0006F5F862F90E08217930708F340E050E0DE
:1001B000C801B7010E943008932F80917A008F7791
:1001C00080937A00ED2DF0E0EE0FFF1FED56FE4F0D
:1001D000822F808331831F910F91FF90EF90DF90EA
:1001E0000895CF93DF93982F6630C8F58A528135F2
:1001F00018F0A0E0B0E00CC0913608F09F7D9A5254
:10020000E92FF0E0EE0FFF1FE45AFF4FA591B491E4
:10021000862F90E0EC01C170D07060FD02C090EFBD
:1002200001C09FE0669570E0695A7E4F20E030E0A3
:10023000FB01E20FF31F4A2F4F7084E0B695A7959C
:100240008A95E1F7209711F04295407F80818923BC
:10025000482B40832B5F3F4F2431310549F7DF9115
:10026000CF91089581118FEF20E030E0F901E95A34
:10027000FE4F80832F5F3F4F24313105B9F708953A
:1002800080E00E943201A7EEB0E08C918F608C93E9
:1002900087EB8093E50087E08093E600E4EEF0E0F2
:1002A00080EC80838081886080838C91806E8C93C9
:1002B0001092520108951F920F920FB60F921124BF
:1002C000EF92FF920F931F932F933F934F935F9360
:1002D0006F937F938F939F93AF93BF93CF93DF934E
:1002E000EF93FF9300910001015000930001809172
:1002F0005601882381F0002381F4809153018823E3
:1003000021F481E08093520108C080915301815013
:100310008093530102C01092840180915201813078
:1003200009F052C0E0905401FF2410E0C0E0D0E09A
:100330006C2F80918401992787FD90958C0F9D1FCC
:1003400097FD15C0112399F4E0918401FF27E7FD83
:10035000F095EC0FFD1FE559FE4F8081F82EFF1C34
:10036000FF24FF1C8F7721F41C2F1F5F01C080E248
:10037000FF2021F094E09E1508F480E20E94F10035
:100380002196C630D105A1F6ACEEB0E0FD01E559ED
:10039000FF4F80818D9381E0A030B807B9F780913D
:1003A0005501882321F081E08093F40002C010926F
:1003B000F400113011F48AEF03C0809184018F5F43
:1003C0008093840110925201002319F483E08093FA
:1003D0000001809154018A3019F41092540105C033
:1003E000809154018F5F80935401FF91EF91DF91D1
:1003F000CF91BF91AF919F918F917F916F915F91BD
:100400004F913F912F911F910F91FF90EF900F907F
:100410000FBE0F901F901895BC0180915201882348
:10042000E1F720E030E006C0F901E559FE4F808396
:100430002F5F3F4F422FFB01E20FF31F8081882384
:1004400019F02931310581F7E42FF0E0E559FE4F2D
:100450001082473048F081E0809356011092840169
:1004600083E08093530104C01092560110928401DE
:1004700081E080935201089580E090E020E2FC0149
:10048000E559FE4F2083019689319105C1F71092FD
:100490006B010895809355010895982F8091520122
:1004A0008823E1F7609356011092840190935201E2
:1004B0000895109254010895893128F4E82FF0E04E
:1004C000E559FE4F608308956F927F928F929F92BD
:1004D000AF92BF92CF92DF92EF92FF920F931F9352
:1004E000DF93CF9300D000D000D0CDB7DEB75B0153
:1004F0006C0120E43EE745E050E00E9430083901FD
:100500004A01B90180E090E020EC31E84AEF5FEF6A
:100510000E94FD077B018C01EA0CFB1C0C1D1D1DBC
:10052000C801B70120E737E140E050E00E94300801
:1005300059016A0180E797E19C012A9DC0012B9D2A
:10054000900D3A9D900D1124A0E0B0E0E81AF90A50
:100550000A0B1B0BC801B70124E630E040E050E075
:100560000E94300889019A01C3016AE070E00E948C
:100570001C086983C3016AE070E00E941C088A833A
:10058000C5016AE070E00E941C086B83C5016AE047
:1005900070E00E941C088C83C8016AE070E00E9431
:1005A0001C086D83C8016AE070E00E941C088E83FD
:1005B00020E030E0AE014F5F5F4FFA01E20FF31F22
:1005C0008081805DF901E559FE4F80832F5F3F4FA9
:1005D0002630310591F710927101809152018823E4
:1005E000E1F7109256011092840181E0809352014C
:1005F00026960FB6F894DEBF0FBECDBFCF91DF9128
:100600001F910F91FF90EF90DF90CF90BF90AF9030
:100610009F908F907F906F900895EF92FF920F932D
:100620001F93DF93CF93CDB7DEB769970FB6F894DA
:10063000DEBF0FBECDBFFE01B296619171918E01FA
:100640000F5F1F4FC801AF010E944105F82EE92E30
:10065000C8010E940C028F2D9E2D69960FB6F8944A
:10066000DEBF0FBECDBFCF91DF911F910F91FF90E5
:10067000EF90089506C020E000002F5F2D37E1F7CE
:1006800001970097C1F7089580E88093610083E0A7
:10069000809361001092700088E08093B60088EC2F
:1006A0008093B30010926E0081E08093810080936C
:1006B000B0002091B6008091B60090E084709070F8
:1006C00030E021703070822B932B892B91F788EECC
:1006D00093E00E943A034FEF51E0F89446BB47BBCA
:1006E00010928500109284001092B200B99BFECF48
:1006F000109281007894B09917C0909184008091F5
:100700008500382F20E0B901690F711DCB0178E118
:100710008B36970724F080916600815008C0885E70
:10072000974114F081E006C0809166008F5F80934E
:10073000660080E050938100882379F208950E943A
:100740004403E1E6F0E080E8808383E080830E9458
:10075000F3038CE090E00E9425040E94400185B7DD
:10076000806885BF85B7806885BF88E090E09093FA
:1007700088018093870184E690E0909386018093BE
:1007800085018FEF9FEFAFEFBFEF809389019093CB
:100790008A01A0938B01B0938C0110928D0110926D
:1007A0008E0110928F01109290011092920110927E
:1007B000910108950E949F03789482E091E00E9445
:1007C0000C0200D088E091E0EDB7FEB79283818300
:1007D0000E944C040F900F9088EE93E00E943A0321
:1007E0000E94CA05FDCF239A82E080936E0086E2C4
:1007F00087BD8CE084BD08951F920F920FB60F92B3
:1008000011248F939F93AF93BF9380918D0190910B
:100810008E01A0918F01B09190010196A11DB11D93
:1008200080938D0190938E01A0938F01B0939001DE
:1008300085B198E0892785B9BF91AF919F918F913C
:100840000F900FBE0F901F9018959093C500809346
:10085000C4001092C00088E18093C10086E08093BC
:10086000C2000895982F2E9A8091C00085FFFCCF7A
:100870009093C60008952F9A8091C00087FFFCCF07
:100880008091C60008958091C00087FD02C080E07D
:1008900008958091C60008950F931F93DF93CF931F
:1008A000CDB7DEB7C055D0400FB6F894DEBF0FBE4F
:1008B000CDBFFE01E95AFF4F619171918E010F5F2B
:1008C0001F4FC801AF010E944105382FF80108C031
:1008D0002E9A8091C00085FFFCCF2093C6003196F0
:1008E00020812223A9F7832FC05BDF4F0FB6F89436
:1008F000DEBF0FBECDBFCF91DF911F910F91089545
:100900008F929F92AF92BF92CF92DF92EF92FF921F
:100910001F93CF93DF934C016A017B014115510571
:100920006105710519F080E090E020C080E3F401DA
:100930008083118241E050E03DC0C701B6012AE04A
:1009400030E040E050E00E943008162FC701B601A9
:100950002AE030E040E050E00E943008C901DA01AE
:100960006C017D01105DF5011083CE015401A80ECC
:10097000B91EEC012196FAE0CF16D104E104F1048E
:10098000E0F68C2D805DF5018083AE01BE0175958A
:100990006795D40120E030E007C09C9180818D9361
:1009A00090832F5F3F4F319726173707B4F3C80D59
:1009B000D91D1882CA01DF91CF911F91FF90EF904E
:1009C000DF90CF90BF90AF909F908F9008950F933E
:1009D0001F93CF93DF938C019B016115710519F073
:1009E00080E090E016C080E3F8018083118241E04E
:1009F00050E02FC0C9016AE070E00E941C08482F37
:100A0000C9016AE070E00E941C089B01405D4083C0
:100A1000CE01F801E80FF91FEC0121962A303105CB
:100A200048F7822F805D8083AE01BE017595679582
:100A3000D80120E030E007C09C9180818D939083A5
:100A40002F5F3F4F319726173707B4F3C00FD11FE1
:100A50001882CA01DF91CF911F910F91089520E074
:100A600030E003C0EC932F5F3F4FFB01E20FF31F19
:100A7000E081DC01A20FB31FEE23A1F71C92C90194
:100A80000895AF92BF92CF92DF92EF92FF920F93B1
:100A90001F93CF93DF937C015B01DA01C0E0D0E0CC
:100AA000CC24DD244FC0853209F044C081818936D1
:100AB00081F08A3628F4833691F1843639F409C0FE
:100AC000833711F1853729F08C3671F0CFEFDFEFE6
:100AD00044C08D010E5F1F4F6D917C91C7018C0F3B
:100AE0009D1F0E94E7040CC08D010C5F1F4F4D91AC
:100AF0005D916D917C91C7018C0F9D1F0E948004B8
:100B0000C80FD91FD80112C08D010E5F1F4F6D9104
:100B10007C91C7018C0F9D1F0E942F05F1CFF7011B
:100B2000EC0FFD1F8C918083219612960894C11CB6
:100B3000D11C05C0F701EC0FFD1F8083219608949E
:100B4000C11CD11CF501EC0DFD1D8081882309F02D
:100B5000AACFEC0EFD1EF7011082CE01DF91CF91DE
:100B60001F910F91FF90EF90DF90CF90BF90AF90CB
:100B70000895DF93CF93CDB7DEB79E01275F3F4F38
:100B80008D819E816F817885A9010E944105CF9159
:100B9000DF910895AF92BF92CF92DF92EF92FF92D2
:100BA0000F931F93DF93CF93CDB7DEB72A970FB67E
:100BB000F894DEBF0FBECDBF83E20E9432040E94D4
:100BC0003B04C82E84E191E00E940C028C2D0E940F
:100BD0003204DD245E010894A11CB11CED2CFF241D
:100BE0000E943B0485010E0D1F1DD8018C930E94AD
:100BF0003204F80100810D3049F00E3018F40A304B
:100C000049F404C0003239F00B3321F4EA0CFB1C28
:100C1000D7011C92D394ED2CFF2487010150104082
:100C2000F501E00FF11F8081882319F0B9E0BD15AF
:100C3000A8F600D08AE191E0EDB7FEB792838183F8
:100C40000E944C04FE0131960E0F1F1F0F900F9053
:100C5000D8018C91882379F08DE191E00E940C02FB
:100C600000D08FE191E0EDB7FEB7928381830E94BF
:100C70004C048FEF2DC0EE0DFF1D1082F4E6CF1651
:100C800091F0FC1520F08DE0C816A1F406C0A0E795
:100C9000CA1631F0B2E7CB1669F4ECEAF6E005C00B
:100CA000EEE1F7E002C0EBE7F6E0CE010196099530
:100CB000882381F08DE191E00E940C0200D08FE149
:100CC00091E0EDB7FEB7928381830E944C048EEFD2
:100CD0000F900F902A960FB6F894DEBF0FBECDBFCF
:100CE000CF91DF911F910F91FF90EF90DF90CF9008
:100CF000BF90AF900895FC018081882349F0CF0117
:100D00000E94520890939201809391010E94A8073B
:100D100000D000D083E291E0EDB7FEB792838183EB
:100D20008091910190919201948383830E944C045D
:100D30008EE291E0EDB7FEB79283818380919101BD
:100D400090919201948383830E940D030F900F90E2
:100D50000F900F9080E00895EF92FF920F931F93F2
:100D6000CF93DF938C01DC018C91882331F0E80173
:100D700095E3E92E91E0F92E2EC010E0C5E3D1E015
:100D8000812F0E94830000D000D0EDB7FEB7D28340
:100D9000C183948383830E944C041F5F0F900F9044
:100DA0000F900F90183061F734C080530E94830079
:100DB00000D000D0ADB7BEB71296FC92EE9211975C
:100DC00014969C938E9313970E944C0421960F9037
:100DD0000F900F900F908881882339F700D000D0B2
:100DE00089E391E0EDB7FEB792838183D801EC915E
:100DF000F0E0EE0FFF1FED5CFE4F80819181EDB7BB
:100E0000FEB7948383830E940D030F900F900F9081
:100E10000F9000D08CE391E0ADB7BEB712969C93D3
:100E20008E9311970E944C040F900F9080E0DF91F9
:100E3000CF911F910F91FF90EF900895CF92DF9285
:100E4000EF92FF920F931F93CF93DF93EC0100D0AB
:100E50008FE391E0EDB7FEB7928381830E944C044B
:100E60000F900F9088E491E00E940C02EE24FF2482
:100E700087012DE4C22E21E0D22E10928D01109216
:100E80008E0110928F011092900100D000D000D0FE
:100E9000EDB7FEB7D282C182E382F4820583168366
:100EA0000E944C048DB79EB706960FB6F8949EBF6D
:100EB0000FBE8DBFCE010E94AC068881882319F039
:100EC0008981843761F481E00E944A02C801B70138
:100ED0000E94640204C00E944304882329F52091E3
:100EE0008D0130918E0140918F0150919001809140
:100EF000850190918601A0E0B0E0281739074A07E4
:100F00005B0748F3E20EF31E041F151F8091890151
:100F100090918A01A0918B01B0918C01E816F9069D
:100F20000A071B0708F4A9CF80E00E944A0280E06C
:100F3000DF91CF911F910F91FF90EF90DF90CF90B5
:100F400008958FEB84B98FEF85B986E585B908954B
:100F5000AC018FEB84B98FEF85B986E585B92B9904
:100F6000FECF85B1866085B92B9BFECF2B99FECF36
:100F7000299828982B9BFECF2B99FECF289A2B9B44
:100F8000FECF2B99FECF80E14030580724F02898FF
:100F90005595479501C0289A2B9BFECF2B99FECFE4
:100FA000289A2B9BFECF2B99FECF2BE030E0CA0175
:100FB000022E02C0959587950A94E2F780FD02C043
:100FC000289801C0289A2B9BFECF2B99FECF215049
:100FD00030408FEF2F3F380751F7299A2B9BFECFD8
:100FE0002B99FECF2A982B9BFECF2B99FECF2A9AC6
:100FF0002B9BFECF2B99FECF0895629FD001739F4C
:10100000F001829FE00DF11D649FE00DF11D929FA4
:10101000F00D839FF00D749FF00D659FF00D9927E3
:10102000729FB00DE11DF91F639FB00DE11DF91F07
:10103000BD01CF0111240895AA1BBB1B51E107C0BC
:10104000AA1FBB1FA617B70710F0A61BB70B881F58
:10105000991F5A95A9F780959095BC01CD010895E7
:10106000A1E21A2EAA1BBB1BFD010DC0AA1FBB1FAC
:10107000EE1FFF1FA217B307E407F50720F0A21B1E
:10108000B30BE40BF50B661F771F881F991F1A948B
:1010900069F760957095809590959B01AC01BD01B5
:1010A000CF010895FC0188279927E89421912032E7
:1010B000E9F3293010F02E30C8F32B3241F02D32F5
:1010C00039F4689404C00E947008820F911D219128
:1010D00020532A30C0F31EF4909581959F4F0895B8
:1010E0007AE0979F902D879F802D910D1124089570
:0410F000F894FFCFA2
:1010F400030F68656C6C6F000D0A232068656C6CC7
:101104006F0D0A00696E707574000D0A003F003F90
:101114000D0A0023204441432025690D0A0044415F
:101124004320256900256920002569000D0A002354
:1011340020706F6C6C0D0A00706F6C6C00256C2055
:021144000000A9
:00000001FF
